:100000003BC0A6C154C053C052C051C050C04FC025
:100010004EC04DC04CC04BC04AC049C048C047C08C
:1000200046C045C044C0040309041C0377007700A0
:1000300077002E00660069007300630068006C00A2
:100040002E00640065000E0355005300420061005D
:100050007300700012011001FF000008C016DC05DB
:1000600003010102000109021200010100801909C7
:10007000040000000000000011241FBECFE5D4E002
:10008000DEBFCDBF10E0A0E6B0E0E6E1FFE002C0D9
:1000900005900D92A236B107D9F710E0A2E6B0E0C4
:1000A00001C01D92A73AB107E1F7C7D432C7A8CF64
:1000B00085B7836085BF8BB780648BBF08951F931E
:1000C000CF93DF9360918800635067FD13C08091E8
:1000D0008500CCE0D0E0C81BD109C457DF4F809128
:1000E00084008D3209F462C08091620087FD84C073
:1000F000109288008091600084FF4AC06091610086
:100100006F3F09F445C0693070F168506093610039
:100110008091780098E889278093780068E0809142
:10012000620087FD8BC0209186003091870086FF9A
:100130006DC0A9E7B0E080E090E0F901E80FF91F99
:10014000E491ED9301966817C1F76150862F90E016
:100150006F5F0196820F931F9093870080938600B4
:10016000162F1C5F0BC0109261008091780098E8F8
:10017000892780937800662391F614E089E790E060
:10018000E3D01C3019F08FEF809361001093600072
:1001900094E186B3837031F49150D9F710928900BD
:1001A00010928300DF91CF911F910895683009F07C
:1001B0009FCF83EC809378008AE580936000109253
:1001C00062008881807659F59A8110928100898138
:1001D000882309F043C01092820022E081E890E079
:1001E00090938700809386008F81882319F49E81E5
:1001F000921708F1922F1FC0CE0130D48F3F51F1DA
:10020000882309F475CF1092610072CF962FD9011F
:10021000E9E7F0E08D9181939150E1F796CFCE011F
:100220000FD5282F8F3F01F7888187FD25C09FEFCD
:1002300080E880936200909361005ACF89E790E054
:10024000AFD4682F893008F453C08FEF80936100DA
:100250001EE19CCF8EE1809360004ACF853071F023
:10026000863091F0883031F1893061F18A3031F196
:1002700020E081E890E0B4CF9E81DACF90938900AE
:1002800020E081E890E0ACCF8B81813049F1823071
:10029000F9F0833029F020E080E480936200A4CF5D
:1002A000992349F586E290E0909387008093860039
:1002B00024E0F2CF21E08BE890E092CF21E081E8CA
:1002C00090E08ECF90938B0020E081E890E088CF83
:1002D00086E690E0909387008093860022E1DCCF51
:1002E00084E590E0909387008093860022E1D4CF4C
:1002F000182F1C5F43CF913051F0923061F686E4A5
:1003000090E090938700809386002EE0C5CF8AE22C
:1003100090E090938700809386002CE1BDCFA82FBA
:10032000B92F80E090E041E050EA60956F5F58F4AB
:100330002D9138EF82279795879510F08427952780
:100340003F5FC8F3F3CF0895EADF8D939D9308953F
:10035000CF93CFB7CF93C395B09BE9F7B09B09C0BC
:10036000B09B07C0B09B05C0B09B03C0B09B01C051
:10037000A1C0DF93C0918500DD27C457DF4FB09B3C
:1003800002C0DF91EBCF2F930F931F9306B32FEF94
:1003900000FB20F94F933F9316B34FEF012700FB6B
:1003A00021F93BE031C04E7F012F16B3216028C0F8
:1003B000102F4D7F2260000006B329C04B7F2460C0
:1003C000012F000016B32BC016B3477F28602AC048
:1003D0004F7E06B320612CC04F7D16B320622FC024
:1003E0004F7B06B3206432C0422706B349934FEFD8
:1003F0000000102710FB20F916B31370C9F1297FF4
:1004000091F2012700FB21F906B3237F89F23150D5
:1004100058F1102710FB22F916B3277E79F2012735
:1004200000FB23F92F7C81F206B3102710FB24F97F
:100430002F7971F200C016B3012700FB25F92F7345
:1004400059F200C006B3102710FB26F9223040F203
:1004500000C016B3012700FB27F9243028F64F7798
:10046000206816B30000F9CF10E41ABF002717C0A8
:100470003B503195C31BD04010E41ABF0881033CA8
:10048000E9F00B34D9F0209183001981110F121378
:10049000EDCF093641F10D3211F0013E39F70093ED
:1004A0008A003F914F911F910F912F91DF91CAB711
:1004B000C6FD51CFCF91CFBFCF91189520918A0023
:1004C000222379F310918800112311F5343012F1B1
:1004D0003093880020938400109185003BE0311B0D
:1004E0003093850017C00091880001308CF40AE534
:1004F0003091600034FD10C000936000C8E7D0E088
:100500000FC02795A8F45150A9F4220F0000F9CF8D
:100510004AE503C042ED01C0432FC4E1D0E032E020
:1005200017B31360C09A17BB08B320E413E05F93BE
:10053000012756E008BB279520F4515021F4220FE3
:10054000F9CF012756E000003B5A08BBD0F22795AF
:1005500028F4515029F4220F0000F9CF012756E06A
:10056000279508BB20F4515021F4220FF9CF012721
:1005700056E02991332308BB21F60C7F10918900A6
:10058000110FC651D04008BB11F01093830010E446
:100590001ABF016017B31C7F402F4C7F5F9100C0D2
:1005A00000C008BB17BB48BB7CCF8091A5008DB9AC
:1005B0008091A2008EB90895282F8823A1F0883059
:1005C00008F03FC089E793E09093A4008093A300D4
:1005D000243001F12530A0F0263081F1263050F191
:1005E0002730E1F008958AE993E09093A400809386
:1005F000A30082E58093A50081E08093A200089586
:100600002230A1F0233070F4213061F780EC809328
:10061000A600089588E18093A600089583E0809362
:10062000A600089580E38093A600089580E6809355
:10063000A60008958CE08093A60008952093A6005C
:1006400008958AE993E09093A4008093A300109208
:10065000A200293041F02A3050F4283051F683E5C9
:100660008093A500089582E58093A50008952B301E
:1006700031F02C3009F0BDCF81E08093A20081E5FC
:100680008093A500089522B79091A60082B7821B9F
:100690008917E0F30895C49AA59AAD9887B38C6240
:1006A00087BBC298C59892B72091A60082B7891BD4
:1006B0008217E0F3C29A92B782B7891B8217E0F3E0
:1006C000C2988091A3009091A4008A59934009F0A8
:1006D00008958091A5008DB98091A2008EB90895EA
:1006E00087B3837D87BB88B3837D88BBA5981DB8FE
:1006F0000895582F2091A60040E030E057FD16C025
:10070000C398440FB4994F5FC59A92B782B7891BBB
:100710008217E0F3C59892B782B7891B8217E0F37E
:100720003F5F383029F0550F57FFEACFC39AE9CF22
:10073000842F08958FB9779BFECF8FB108950F93C3
:100740001F930FE1E091A300F091A4008CEA0995BA
:10075000E091A300F091A40083E50995E091A30046
:10076000F091A40080E00995182FE091A300F0918A
:10077000A40080E00995133539F11DB892B7209196
:10078000A60082B7891B8217E0F3C59A92B782B799
:10079000891B8217E0F3C598E091A300F091A400B3
:1007A00083E0EA39F80721F0002351F00150CECF61
:1007B0008091A5008DB98091A2008EB90023B1F778
:1007C00081E01F910F91089580E01F910F9108958E
:1007D000EF92FF920F931F937B018C01862F817004
:1007E000880F880F880FE091A300F091A400806229
:1007F0000995D801C70129E0B695A79597958795E2
:100800002A95D1F7E091A300F091A40009951695DF
:100810000795F794E794E091A300F091A4008E2D42
:100820000995E091A300F091A40080E009951F9143
:100830000F91FF90EF9008950F931F938C01E0911B
:10084000A300F091A40080EA0995E091A300F09143
:10085000A400812F0995E091A300F091A400802FBE
:100860000995E091A300F091A40080E009951F9103
:100870000F910895FF920F931F938C01F62EE09134
:10088000A300F091A40080EC0995E091A300F09101
:10089000A400812F0995E091A300F091A400802F7E
:1008A0000995E091A300F091A4008F2D09958EE1A8
:1008B000B7D080E01F910F91FF900895CF92DF9203
:1008C000EF92FF920F931F936B017C01142FE09125
:1008D000A300F091A4008CE40995D701C60149E07A
:1008E000B695A795979587954A95D1F7E091A3007E
:1008F000F091A4000995D701C601B695A7959795E3
:100900008795E091A300F091A4000995E091A300E0
:10091000F091A40080E009951F3FF1F012B70EE1BD
:10092000C701B60155DF8F3F79F482B7811B8D3344
:10093000B8F312B70150A1F781E01F910F91FF901A
:10094000EF90DF90CF90089580E01F910F91FF907E
:10095000EF90DF90CF9008958FE062D080E01F91FC
:100960000F91FF90EF90DF90CF900895CF92DF929C
:10097000EF92FF920F931F936B017C01042F122FB4
:10098000862F8170880F880F880FE091A300F09167
:10099000A40080640995D701C60169E0B695A795C2
:1009A000979587956A95D1F7E091A300F091A400FF
:1009B0000995D701C601B695A79597958795E091BA
:1009C000A300F091A4000995E091A300F091A40088
:1009D000802F09951123C1F00F37F1F012B70EE106
:1009E000C701B601F5DE8F3779F482B7811B8D33ED
:1009F000B8F312B70150A1F781E01F910F91FF905A
:100A0000EF90DF90CF90089580E01F910F91FF90BD
:100A1000EF90DF90CF9008958FE002D080E0F5CF87
:100A2000382F882349F020E092B782B7891B8C3396
:100A3000E0F32F5F2317C0F3089512BA18BA8BEFB3
:100A400081BB8FEF87BB17BA93E094BB8EEF85BB5A
:100A500093BF2EDB789433DB32DBFDCFFF920F9315
:100A60001F93CF93DF93F82E292F062F4091630019
:100A7000413051F0443041F01FEF812FDF91CF9191
:100A80001F910F91FF900895002309F487C08F2DC7
:100A9000922F9C01E90110E053C080917400909165
:100AA0007500892B09F058C0609170007091710039
:100AB000809172009091730021E0488157DF80910E
:100AC00064009091650001979093650080936400A5
:100AD000892BD9F4109263008091760081FF3AC08F
:100AE0008091770090E0209174003091750082171A
:100AF000930781F160917000709171008091720094
:100B0000909173004881DADE11E08091700090913D
:100B10007100A0917200B09173000196A11DB11DEA
:100B20008093700090937100A0937200B093730053
:100B300021969E012F19201708F09FCF4091630046
:100B4000413009F4AACF68818091700090917100C2
:100B500091DEB5CF11E0D9CF609170007091710036
:100B6000809172009091730020E04881FFDE8091B7
:100B70007700815080937700882309F0A0CF60919F
:100B800070007091710080917200909173004881A3
:100B900095DE809174008093770091CF10E06DCF47
:100BA0000F931F93CF93DF93082F162F409163006D
:100BB000842F8250823038F01FEF812FDF91CF9148
:100BC0001F910F910895662399F1802F9C01E901EF
:100BD00020C080917000909171002EDE88838091FA
:100BE000700090917100A0917200B0917300019615
:100BF000A11DB11D8093700090937100A0937200AD
:100C0000B093730021969E01201B211778F4409128
:100C100063004230F1F66091700070917100809134
:100C2000720090917300D4DD8883D9CF183028F6F4
:100C300010926300812FDF91CF911F910F91089542
:100C40000F931F93CF93DF938C01EC018981813047
:100C5000F1F0823009F4BCC0833091F1843009F4A2
:100C60008EC0873009F462C0853009F42DC186300A
:100C700009F4E6C0883009F4B4C0893009F42BC106
:100C80008A3009F43CC180E0C8E6D0E043C0A398B4
:100C9000AB9A000000009B9BA1C0A29AAA980000FA
:100CA00000009B9B40C08091660086DCA298AA9AB7
:100CB00010926700A998EFDC80E0C8E6D0E02AC077
:100CC000E091A300F091A400E8018A810995C8E6AB
:100CD000D0E0809368002091A3003091A400F80137
:100CE0008381F9010995809369002091A3003091D7
:100CF000A400F8018481F901099580936A0020918C
:100D0000A3003091A400F8018581F9010995809331
:100D10006B0084E0D0938700C0938600DF91CF9171
:100D20001F910F91089588E047DCC0CF8091670044
:100D3000882399F4E8019B8180E02A8130E0822BAE
:100D4000932BAA2797FDA095BA2F809370009093BC
:100D50007100A0937200B0937300F801978180E056
:100D6000268130E0822B932B909365008093640062
:100D700083E0809363008FEFC8E6D0E0CBCF809113
:100D80006700882399F4E8019B8180E02A8130E0A4
:100D9000822B932BAA2797FDA095BA2F80937000E2
:100DA00090937100A0937200B0937300F801978143
:100DB00080E0268130E0822B932B90936500809316
:100DC000640082E0809363008FEFC8E6D0E0A2CF9A
:100DD00087DCA99A80E0C8E6D0E09CCF89E0ECDB14
:100DE00067CF80916700882399F4F801938180E0B0
:100DF000228130E0822B932BAA2797FDA095BA2F52
:100E00008093700090937100A0937200B093730070
:100E1000109275001092740010927600E8019F8184
:100E200080E02E8130E0822B932B9093650080939D
:100E3000640084E0809363008FEFC8E6D0E06ACF5F
:100E400080916700882399F4E8019B8180E02A81E2
:100E500030E0822B932BAA2797FDA095BA2F809381
:100E6000700090937100A0937200B0937300F8012A
:100E700084819581292F2F7020937600492F50E08F
:100E8000407F507042955295507F5427407F5427A1
:100E9000480F511D509375004093740020FF02C00D
:100EA00040937700E8019F8180E02E8130E0822B23
:100EB000932B909365008093640081E0809363009E
:100EC0008FEFC8E6D0E026CF3ADCC8E6D0E08093CA
:100ED000680081E01FCF81E080936700F801828184
:100EE0009381A481B5818093700090937100A09349
:100EF0007200B093730080E0C8E6D0E00BCFE80149
:100F00008A8180936600C8E6D0E01092680081E094
:060F100001CFF894FFCFB1
:020F16005AFF80
:00000001FF
